:020000020000FC
:1000000012C01895189518951895189559C01895F7
:1000100018955CC018951895189518951895189509
:100020001895189518951FE524E01DBF2EBF599807
:100030001FE219B918E11AB911E119BF00240FBC68
:100040000EBC03BE789438D0CC27533008F4C4607B
:1000500051FFC1601124222402BE0DBC0CBCE2EA97
:10006000F0E0152F110FE10FF01D159125912BBD1B
:100070001ABD17E02DE02EBD13BFC1FFFECFC0FD9E
:1000800003C0C160CD7FF9CFC2FD02C0212C12B6E2
:10009000C3FD5068152F0CD0112D0AD0122D08D099
:1000A000D2CFD002201CA08C0000D002201CA08C3B
:1000B0005D9BFECF1CB908955F9BFECF5CB1089598
:1000C000C0FF02C003BE0EBCC2601895139439F481
:1000D000C2FD02C0C8601895239409F4C860189541
:00000001FF
